:020000040800F2
:100000000804002005010008290100082B01000850
:100010002D0100082F010008310100080000000038
:100020000000000000000000000000003301000894
:100030003501000800000000370100083901000800
:100040003B0100083B0100083B0100083B010008A0
:100050003B0100083B0100083B0100083B01000890
:100060003B0100083B0100083B0100083B01000880
:100070003B0100083B0100083B0100083B01000870
:100080003B0100083B0100083B0100083B01000860
:100090003B0100083B0100083B0100083B01000850
:1000A0003B0100083B0100083B0100083B01000840
:1000B0003B0100083B0100083B0100083B01000830
:1000C0003B0100083B0100083B0100083B01000820
:1000D0003B0100083B0100083B0100083B01000810
:1000E0003B0100083B0100083B010008DFF810D08D
:1000F00000F02EF800480047A5030008AFF3008089
:10010000080400200D488047DFF83400016841F4FE
:10011000E0210160BFF34F8FDFF82800DFF82810DF
:1001200001600A4800477047FEE7FEE7FEE7FEE78A
:10013000FEE7FEE7FEE7FEE7FEE7FEE72701000831
:1001400024ED00E00CED00E00003FA05ED000008EE
:10015000064C074D06E0E06840F0010394E8070014
:1001600098471034AC42F6D3FFF7C4FFE803000809
:100170000804000870B5194C8320206000256560D4
:10018000A56017486060012000F02EF86168084300
:10019000606014490D60086840F002000860206843
:1001A00040F48030206020688003FCD5206840F057
:1001B0008070206020688001FCD5606820F003001A
:1001C0006060606840F002006060606840F4800039
:1001D0006060086840F01000086070BD00100240C8
:1001E00000841D0000200240012804D0B0F5807F6B
:1001F00003DD012102E000202CE00021802801DD48
:10020000012200E000220A44402801DD012100E033
:1002100000210A44102801DD012100E000210A44E8
:10022000082801DD012100E000210A44042801DD45
:10023000012100E000210A44022801DD012100E043
:1002400000211144012801DD012000E000200844C4
:10025000C01D0001702800D100207047012181409D
:100260000148016070470000140C014001218140E9
:100270000148016070470000100C0140F0B53B4E92
:100280003B4CB04203D1A66946F00406A661394E44
:10029000B04203D1A66946F00806A661364EB042C8
:1002A00003D1A66946F01006A661344EB04203D1D0
:1002B000A66946F02006A661314EB04203D1A66978
:1002C00046F04006A66100240F2900DD0124692ABA
:1002D00001D0492A02D1032B00D10124032B00DDD8
:1002E0000124692A06D0492A04D06F2A02D04F2A55
:1002F00000D00124692A01D0492A00D100256F2AA3
:1003000001D04F2A00D1012503260222082915DA3F
:10031000076802EB810206FA02FC27EA0C07076075
:10032000076893401F430760026889008E40B2430C
:10033000026002688D402A43026015E00839476870
:1003400002EB810206FA02FC27EA0C0747604768C5
:1003500093401F434760426889008E40B243426029
:1003600042688D402A4342602046F0BD00080140AB
:1003700000100240000C0140001001400014014038
:100380000018014002E008C8121F08C1002AFAD173
:1003900070477047002001E001C1121F002AFBD105
:1003A00070470000FFF7E6FE00236F220121074897
:1003B000FFF764FF09E000F00BF80120FFF756FF9C
:1003C00000F006F80120FFF749FFF4E7000C0140B8
:1003D000034804490160016801390160FBD170479D
:1003E00000000020A0BB0D00080400080000002051
:1003F00004000000840300080C040008040000202E
:0C04000004040000940300080000000049
:04000005080000ED02
:00000001FF
